:020000008C284A
:1000080009008A014408C40A82073A341B34222AA8
:100018008534CA34602A4634BA34272945346234D0
:100028001829E234BB3478290F34E834FD290D341B
:10003800A334EE289434B9340529D23499340329E9
:10004800F03453342429A634383409291934F234C5
:1000580010299D34C23449299F340334122A9B3411
:1000680008343829003400348A0182000D340A34F7
:100078005334503459344434413452343E340034C7
:100088000D340A34563465347234733420343234BF
:100098002E3432343A3420344534633468346F347F
:1000A8003D340034203454347234693467343D3478
:1000B8000034203444346C3479343D3400342034F2
:1000C80041346E3461343D3400344F344E3400349E
:1000D8004F344634463400340D3445347234613478
:1000E800733465343A3420340034203428344134AD
:1000F80062346F3472347434293400348A018207CC
:100108000F3400340E3401340C34033408340B3407
:100118008316333085000730870000309000863022
:10012800810050309F0091018312043092001E30EC
:10013800B800BD014C21F423FA305124871632301F
:100148005124871232305124871CAD28071CB2284D
:10015800A228FA3051248718A228BD28871208300F
:10016800B400FA3051240718A228B40BB528871612
:100178007829FA305124612364305124EE20BD15CA
:10018800BD103D128716C7013A3092223D140B2349
:1001980039233E083F040319E828C4010520C2009A
:1001A8000520C30042040319EA2842083E06031D3D
:1001B800E32843083F06031DE3280520CC28C40A8A
:1001C800D22879309222C3283D1EC32861233F30AC
:1001D8006623C328443092226930291C6C3092224D
:1001E8005D3092222A08B922563092226930A91C21
:1001F8006C309222633092222B08B9220800023018
:1002080006290130C7003D1608003D1EEA284708A8
:10021800A9043D12412108003D1EEA284708FF3A7B
:10022800A9053D124121080061239B22B500003A2F
:10023800031920293508AA002A08B92241210800F3
:1002480060214121080059216123D101D201C6232F
:100258004030D1070318D20A703092223C21BD18D1
:10026800E528D21F2B29080039236123FC22080026
:1002780052080123510801230800D101D2015A3044
:10028800A80069212830B32308004C21EE2008007B
:10029800D101D20128309C2328085A3A031D59213C
:1002A8002C0883169100831208000130AA00A901C6
:1002B800AB016921A914080061239B22B500033C06
:1002C800031CEA283508AB0008002B08B50003100A
:1002D800B50D35088220AD00B50A35088220AC007E
:1002E80083169100831208007A22BD196123B00198
:1002F80087162A08B900BD1D83298718B0290B1D48
:100308007F290B1164308100230803390319810305
:10031800E421BD1AB029B90B7F290508BA212D059A
:10032800B500A91C9A29300603197C293508B000A4
:10033800C621D421C80A0319C90A8712BD1DA829D4
:10034800291CA82938227C292030B3230830D1075A
:100358000318D20AD21F7C292918E528FF30A000EB
:100368002030B323BD19E5288712B829B500B60196
:1003780035183614B518B614351A3615B51AB61513
:1003880036080800B500A401A501A601A701B50C0F
:10039800A40DB50CA50DB50CA60DB50CA70D080040
:1003A8002D18080000308422A400AD180800013080
:1003B8008422A5002D19080003308422A600080015
:1003C800BD12A30A2308643A031D0800A301A20A68
:1003D80022083C3A031D0800A201A10A21083C3A60
:1003E800031D0800A101A00A2008FA3A0319BD1646
:1003F800080061237A22BE01BF0120309C23200817
:10040800FF3A0319102ABF0A0319BE0A0830D10798
:100418000318D20AD21F012AC722080020308400FC
:100428000830BA0061230008840A01235E22BA0B4F
:10043800172A64305124BD180800142A7A22203063
:100448009C232008FF3A0319080038220A30512457
:10045800BD180800C80A0319C90A0830D1070318CB
:10046800D20AD21F232A080061234908BE0048087F
:10047800BF00C7225E222008C1225E222108BD22B9
:100488005E222208BD222E3066232308BD225E226A
:1004980024082D183D115D222508AD183D115D2257
:1004A80026082D193D115D222708AD193D115D2241
:1004B8000800BA222030662BD101D20161232030F6
:1004C8009C230830BA00203084000008840A0123E5
:1004D8005E22BA0B692A64305124BD18080008301E
:1004E800D1070318D20AD21F622A0800A001A1016D
:1004F800A201A3010830D100D201C801C901080036
:100508000739B5000310B50DB50D35089F001F1448
:1005180059249F149F188E2A1E080800CC004C08E6
:100528003820003A031908006623CC0A932AB70139
:100538004823B500203A03199B2AA42A4823B5006A
:100548003030B502031CB02A0A3035020318B02A2D
:10055800B2223508B707A22A370808000310B70DDA
:100568003708B70DB70DB70708003D11BF00BE012A
:10057800D22A3D15BE01BF00D62A3D15BE01BF00D7
:10058800D22A3D11C82A3D152730C0001030C100BD
:10059800E0220330C000E830C100E022C00164302E
:1005A800C100E022C0010A30C100E022C0010130D0
:1005B800C1003D15E02208003030B500EE22031CD2
:1005C800E82A3D15B50AE22AF5223D1D080035083E
:1005D800662308004108BF024008031C400FBE0202
:1005E80008004108BF070318BE0A4008BE070800F4
:1005F8003E0801233F0801230800C600460E0523D4
:1006080046080F39F63E0318073E3A3E662BBB01F3
:1006180079235723BC00BD1808000A3A03190C2B8C
:100628003C08083A0319292B3B08533E84003C0830
:1006380080003D1866233C080D3A0319372BBB0A86
:100648003B08133A0319332B0C2BBB03BB1B0B2B97
:100658000830662320306623083066230C2B0830C8
:100668006623BB030C2BBB010800BE01BF01482356
:1006780003180800BF07BE060310BF0DBE0DBF0D4F
:10068800BE0DBF0DBE0D3B2B3B08533E840000083A
:10069800BB0AB5000D3A0319BB0335082F3C3508D2
:1006A8000800BB0308009F3E031C5F2BE63E0318AF
:1006B800203E5B3E0800613E08000D3066230A308C
:1006C80066230800B700B5000830B30097239723C6
:1006D8000511972337180515371C0511B70C9723F3
:1006E800B30B6E2B0515350808000830B300B701A9
:1006F800871C7C2B8F23871C7C2B97230310B70C1C
:10070800871CB7170000B30B812B97233708BD1040
:100718008718BD1408003808B6000310B60CB603D5
:10072800B603B603992B3808B600B60B992B080008
:1007380084000830BA00E323A030022452080224BF
:1007480051080224E323A1300224AB2B36242324AE
:100758008000840ABA0BAA2B4424F42308008400DE
:100768000830BA00E323A0300224520802245108BA
:10077800022400080224840ABA0BBD2BF423073094
:1007880051240800E323A03002245208022451080F
:1007980002244030B400FF300224B40BCF2BF423E2
:1007A800073051240800E323A03002245208022411
:1007B800510802240800E323A1300224080083160C
:1007C8008711831287110000831607158312000012
:1007D8008715071183160711831200008711080077
:1007E800871107118316071183120000871500006F
:1007F800831607158312000087110800B50008301A
:10080800B300B50D0711831603180715031C07114C
:10081800831200008715000000008711B30B052C18
:100828008316071583120000000087150000071DB6
:10083800202C8711EA140800EA10871108000830F4
:10084800B3008316071583128715000003100719D4
:1008580003148711B50D000000000000B30B282C0D
:1008680035080800071183160711831200000000DD
:100878008715000000000000000000008711080034
:10088800831607158312000000008715000000007A
:1008980000000000000087110800BD10B2005B24B2
:1008A800B20B532C080001305C2C0A305C2C6430ED
:1008B800B10000008718BD148718BD148718BD142F
:1008C8008718BD148718BD148718BD148718BD1460
:0A08D8008718BD14B10B5D2C080059
:02400E00E400CC
:00000001FF
